:020000002B28AB
:08000800CE000308DC008301B7
:10001000B10131148618B1148B105C0883004E08AE
:100020000900820700000A3414341E3428343234A4
:100030003C34463450345A3464346E347834823428
:100040008C349634A034AA34B434BE34C834D23498
:10005000DC34E634F034172604309F00FF3085008E
:10006000033086001230870001178E30920014266C
:10007000B101B901BA01BB01BC018501860187014B
:100080000715DE01BE01C501C4010130BD008B179B
:1000900041309F00A42547309B009D121D129D15E5
:1000A0001D15121592101214E523BE100B125B23BE
:1000B000C81F5728BE143E118B10B1010B1600301B
:1000C0004B21B321071087157E22E8215508C22055
:1000D000CF00E32002245B2303014806031D772899
:1000E00003014906031D77285F18922864280B1224
:1000F000DF01C81F7F2800308B2107155428481BBB
:10010000042BC81A732D481AFA28C8188D284919C3
:10011000A0208B10B1010B1664285F143114B110AC
:10012000DE016428DE0A02305E06031D642807191A
:100130009C28DE01DF018928DE013114B11064281A
:100140008B10B1010B16311CBB28B11CAF28D50395
:10015000FF305506031DB7280030D500B728D50A53
:100160000A305506031DB7280930D500B7285508B1
:10017000C220CF00B101E320022449115B234919B9
:10018000A32808008207F234F034EE34EC34EA3469
:10019000E834E634E434E234E134D801D901D70A52
:1001A000D70BDB283030D807D9075906031D0800C4
:1001B0002030D9000800D80A0A305806031DD0287C
:1001C000D801D90AD0289F15D925D9251F15D92599
:1001D000D9251E08D4004F081E0203190800031871
:1001E000F6284F081E02031CF8280800071508000F
:1001F000071108008B10B1010B163E1500308B2142
:100200000E29BD0A0B303D0601300319BD000E2931
:10021000BD0300303D060A300319BD003D08112022
:100220004B21B922E82102245B23C81B5428481A19
:100230005A28C81922294919A020311C1129B11C9A
:100240000129082900304B213D0811208B210E295E
:1002500087110714DC30D400172687101426B92222
:10026000E821022408004811871507101726871473
:1002700014268B10B10108008711DC30D40007155B
:100280000714B922E82102240800C91187150710B4
:100290008B10B10108001A268D0082213508B800A4
:1002A00082213508B70082213508B6008221350841
:1002B000C20082213508C30082213508C400822192
:1002C0003508C70082213508C60082213508C500DF
:1002D00082213508D5003030C100003044060319B2
:1002E00008004130C10001304406031908004230C3
:1002F000C10002304406031908004330C10044061F
:10030000031908001D268C130C141A268D0A0C08DC
:100310001426B50008001A268D0014263808A321DB
:100320003708A3213608A3214208A3214308A321AB
:100330004408A3214708A3214608A3214508A32177
:100340005508A32108001A268C001D268C130C15B5
:1003500055308D00AA308D008C140C11CB251A2637
:100360008D0A1426080007178717871307138717A6
:100370008713071387178713071387178713071721
:10038000871787130717871787130713871787138D
:1003900007138717871307178717871307138717FD
:1003A00087130713871787130713871787130713F5
:1003B0008717871307138717871307138717871361
:1003C0000717871787138716000000008712080099
:1003D0003908A0003808A1003708A2003608A30099
:1003E0000718FF29F830A3020318FA29A2080319F5
:1003F000A103A203A130A202031CA103A1032308AD
:100400003A06031D0C2A22083B06031D0C2A21086C
:100410003C06031D0C2A08002108BC002208BB0072
:100420002308BA000030A9001930AA007526003050
:10043000A9004030AA00752607132219071787174D
:1004400087130713A2180717871787130713221894
:100450000717871787130713A31B07178717871318
:100460000713231B0717871787130713A31A0717E9
:10047000871787130713231A07178717871307137D
:10048000A319071787178713071323190717871748
:1004900087130713A3180717871787130713231842
:1004A0000717871787130713401B0717871787132B
:1004B0000713C01A0717871787130713401A071760
:1004C000871787130713C019071787178713071391
:1004D00040190717871787130713C01807178717BF
:1004E00087130713401807178717871307138717F2
:1004F000871387160000000087120800311CB92AF4
:10050000B11C9D2A4608B60203188A2AB7080319A7
:10051000B803B7034708B702031CB8031530380601
:10052000031DB92AF93037020318B92A2030B60062
:100530004730B7001630B800B92A4608B607031886
:10054000B70FA32AB80A4708B7070318B80A163026
:100550003806031DB92A47303702031CB92A203058
:1005600036060319B92A0030B600F930B700153045
:10057000B800B101D1222D232D080F39303EAF0034
:100580002C0E0F39303EAE002C080F39303EAD0036
:100590002B0E0F39303EAC002B080F39303EAB002C
:1005A00008008719E02A3E1808003E14013044066E
:1005B0000319EC2A023044060319F92A3E100800F8
:1005C0003E1C08003E10013044060319F92A02308F
:1005D00044060319EC2A08004308B6020318F42A5B
:1005E000B7080319B803B7034208B702031CB803DE
:1005F00008004308B6070318B70FFF2AB80A4208D5
:10060000B7070318B80A0800C40A033044060319E0
:10061000C4010130440603191A2B023044060319A1
:10062000212B033044060319282BC301C2013030AB
:10063000C10089287030C3001730C2004130C100AA
:1006400089287030C3001730C2004230C1008928A9
:10065000C301C2014330C10089282030B000AB0182
:10066000AC01AD01AE01AF010310B60DB70DB80D71
:10067000B90D03183614AB0DAC0DAD0DAE0DAF0DAD
:10068000B003031D442B08002B3084005023840A40
:100690005023840A5023840A5023840A5023342B85
:1006A00003300007CA00CA19800030300007CA00B2
:1006B000CA1B800008009F11D925D925D925D92525
:1006C0001F15D925D9251E08CA00D925D925D92510
:1006D0001F15D925D9251E084A06031D5B2BC80105
:1006E000C9012F301E02031C7B2B36301E0203185B
:1006F0007B2BC817DA2BBE1C080016301E02031C09
:10070000872B1D301E020318872B4817DA2B233046
:100710001E02031C912B2A301E020318912BC816AF
:10072000DA2B48301E02031C9B2B4F301E0203188D
:100730009B2B4816DA2B55301E02031CA52B5C3070
:100740001E020318A52BC815DA2B3C301E02031C11
:10075000B02B43301E020318B02B48152821DA2B8A
:100760007B301E02031CBA2B82301E020318BA2BE8
:10077000C814DA2BC52B62301E02031CC52B69304E
:100780001E020318C52B4814DA2B0A301E02031C64
:10079000D02B10301E020318D02BC9153C21DA2BA8
:1007A0006D301E02031C080076301E02031808007C
:1007B000491508001F15D92506301E020318DA2B2B
:1007C00048193321C919452108000710871106115E
:1007D000D9250130F2250615D9252030F225203003
:1007E000F2252030F2252030F2252030F22520306D
:1007F000F2254F30F2254630F2254630F2252030E2
:10080000F22508000611D9254030F2250615D92514
:10081000E030540203180D2C482CE2305402031827
:10082000122C592C0930DD00E430540203181A2C24
:100830004024692CE63054020318202C40247A2CE2
:100840001130DD00E83054020318282C40248A2C93
:10085000EA30540203182E2C40249B2C1930DD0062
:10086000EC3054020318362C4024AB2CEE305402EA
:1008700003183C2C4024BC2C2130DD004024CC2C1F
:10088000DD0303015D06031908000030F225402C4A
:100890000330F2251B30F2251B30F2251B30F225E8
:1008A0001B30F2251B30F2251B30F2251B30F225C0
:1008B000692C0030F2251830F2251830F225183056
:1008C000F2251830F2251830F2251830F2251830AC
:1008D000F2250030F2250030F2250330F2251B30DE
:1008E000F2251B30F2251B30F2251B30F2251B3080
:1008F000F2258A2C0030F2250030F2250030F22556
:100900001830F2251830F2251830F2251830F2256B
:100910001830F2250030F2250030F2250030F225A3
:100920000030F2250330F2251B30F2251B30F22572
:100930001B30F225AB2C0030F2250030F2250030C0
:10094000F2250030F2250030F2251830F22518305B
:10095000F2251830F2250030F2250030F225003063
:10096000F2250030F2250030F2250030F225033068
:10097000F2251B30F225CC2C0030F2250030F22578
:100980000030F2250030F2250030F2250030F2254B
:100990000030F2251830F2250030F2250030F22523
:1009A0000030F2250030F2250030F2250030F2252B
:1009B0000030F2250330F2250611D9258030F225CA
:1009C0000615D9255430071C5230F2255830F2252F
:1009D00020304819F730F2253130F2253430F22535
:1009E0002F08F2252E08F2252D08F2252C08F225D5
:1009F0002E30F2252B08F2250430F2250330F225A3
:100A00000230F2250130F2250030F2250611D925F9
:100A1000C030F2250615D9257330F2256830F2254D
:100A20002030F2254108F2252030F2252030F22531
:100A30003E19372D7330F2257430F2252030F2251F
:100A400041304507F2252030F2252030F225733061
:100A5000F2257130F2255508D700CD205808DA006C
:100A60005908DB005B08F2255A08F22508006D30B2
:100A7000F2256530F22554255308F2255208F22557
:100A80002030F2252030F2257330F2257130F22526
:100A90005508D700CD205808DA005908DB005B085C
:100AA000F2255A08F2250800D101D201D3013D08F0
:100AB000D100D10AD10B6B2D000003015306031D99
:100AC000642D2030D300662D3030D3073030D2076C
:100AD000000000000800D20A0A305206031D5A2DF9
:100AE000D201D30A5A2DC50A033045060319C501A0
:100AF000013045060319852D0230450603198C2D5A
:100B00007D30C6000030C700892836189C25FA3091
:100B1000C6000030C7008928CA0136184A14B61822
:100B20004A1436194A144A189A2DE830C600033080
:100B3000C70089289C258C2D7D30B607031C080032
:100B4000B70A0319B80A0800CB25061686178612BD
:100B50000613ED25D925ED25D925ED25D925061234
:100B6000ED25D9252830F2250830F2250C30F22564
:100B70000130F225C425860108000730B200643038
:100B8000B300FF30B400E62D0230B2003230B300C3
:100B9000FF30B400E62D0130B2001430B300FF3056
:100BA000B400E62D0130B2002830B300FF30B400AD
:100BB000E62D0130B2000730B3009330B400E62DCB
:100BC0000130B4000130B2000130B300B40BE62DA7
:100BD000B30BE62DB20BE62D08008615E025861135
:100BE000E0250800B5000612351A06168613B51A58
:100BF00086178612351B86160613B51B0617861533
:100C0000E0258611E0250612351806168613B5185C
:100C100086178612351986160613B5190617861516
:100C2000E0258611E0250800031383120800031352
:100C300083160800031783120800031783160800A1
:100C400028262608A8070318A70A2508A70700349E
:100C5000A609A60A0319A503A5090034A301A40146
:100C60002008CB002108CC002208CD000830B000BD
:100C7000AA0C0318492EB00B382EB000A90C03188B
:100C8000472EB00B3E2EA001A101A201003403109B
:100C90006D2E0310582EAA0C031C582E4D08A207C7
:100CA0004C0803184C0FA1074B0803184B0FA00763
:100CB000A00CA10CA20CA30CB00B4B2E0830B00062
:100CC000A90C031C6D2E4D08A2074C0803184C0FED
:100CD000A1074B0803184B0FA007A00CA10CA20CF6
:100CE000A30CA40CB00B602E0800BF01C001CA0108
:100CF000200DC00D2A08C0022908031C290FBF02BD
:100D00000301031C0130CA02A00D0730B000200D02
:100D1000C00DBF0DCA0D2A08201C982EC00229083C
:100D2000031C290FBF020301031C0130CA02A12EBC
:100D3000C00729080318290FBF0703010318013052
:100D4000CA07A00DB00B872E210DC00DBF0DCA0D17
:100D50002A08201CB52EC0022908031C290FBF0237
:100D60000301031C0130CA02BE2EC0072908031864
:100D7000290FBF07030103180130CA07A10D07306F
:100D8000B000210DC00DBF0DCA0D2A08211CD22EA6
:100D9000C0022908031C290FBF020301031C0130F4
:100DA000CA02DB2EC00729080318290FBF07030159
:100DB00003180130CA07A10DB00BC12E220DC00DC2
:100DC000BF0DCA0D2A08211CEF2EC0022908031CE2
:100DD000290FBF020301031C0130CA02F82EC0070D
:100DE00029080318290FBF07030103180130CA0798
:100DF000A20D0730B000220DC00DBF0DCA0D2A088C
:100E0000221C0C2FC0022908031C290FBF0203015A
:100E1000031C0130CA02152FC00729080318290F27
:100E2000BF07030103180130CA07A20DB00BFB2E48
:100E3000230DC00DBF0DCA0D2A08221C292FC00288
:100E40002908031C290FBF020301031C0130CA0239
:100E5000322FC00729080318290FBF070301031801
:100E60000130CA07A30D0730B000230DC00DBF0D20
:100E7000CA0D2A08231C462FC0022908031C290F6B
:100E8000BF020301031C0130CA024F2FC00729080B
:100E90000318290FBF07030103180130CA07A30D68
:100EA000B00B352F23185A2F2A08C007290803181A
:060EB000290FBF07080036
:02400E00313F40
:104200001500F900000000000000000000007D0023
:104210000000020016003700800017007000010047
:1042200000007D0000000200160038007A00170030
:104230007000010000007D0000000200160039003F
:10424000740017007000010000007D0000000200F3
:1042500016003A006E0017007000010000007D009B
:104260000000020016003B0068001700700001000B
:1042700000007D000000020016003C0062001700F4
:104280007000010000007D000000020016003D00EB
:104290005C0017007000010000007D0000000200BB
:1042A00016003E00560017007000010000007D005F
:1042B0000000020016000C00880000000000000052
:1042C00000007D000000020016000E007C000000CF
:0C42D0000000000000007D000000020063
:00000001FF
